:1007F3003F065B4F666D7D077F6F00FEFDFBF7EFE6
:10080300DFBF7F00020005000500010003000600B2
:0B0813000100040007000200050007C0
:10087C001207C41207931206FA12000E12031B126F
:04088C00069780F259
:1006970020A2257F1412082620A21D20A2081200DE
:1006A7000E12031B80F57F0A1208260516E4F50BC8
:1006B700E516B40703E4F51620A11AE51660167FC0
:1006C7000A12082620A10E20A10812000E12031BF1
:1006D70080F512061E20A01AE51660167F0A12087A
:1006E7002620A00E20A00812000E12031B80F51270
:0306F70005932246
:10059300E5166401701215091204898F15E509B473
:1005A300FF0375096312075CE516640270111511E8
:1005B3001204898F15E511700375110C120793E569
:1005C300166403702815121204898F15E512701D25
:1005D300E511B4020D30000575121D801075121C53
:1005E300800B30010575121F800375121EE516B4CA
:1005F300040A1510E510B4FF03751017E516B405CA
:100603000A150EE50EB4FF03750E3BE516B4060A94
:0B0613001508E508B4FF0375083B2242
:10061E00E516640170081204878F1512075CE51643
:10062E006402701205111204898F15E511B40D03C1
:10063E00751101120793E5166403701F051212045B
:10064E00898F15E511B40209E512C3950F400C8090
:10065E0007E512C3950A4003751201E516B4040AA4
:10066E000510E510B41803E4F510E516B4050A05F7
:10067E000EE50EB43C03E4F50EE516B4060A0508C5
:09068E00E508B43C03E4F5082280
:1007C400D202758901758C4CE4F58AD2AFD2A9D2D4
:1007D4008C75090875110B751216751014750E1E9B
:0F07E40012075CE4F516F580C2A5C2A6C2A722D3
:10084600E4F580D2A7F580C2A77580FFD2A59008EF
:0B0856000593F580C2A57F0102082673
:10086100E4F580D2A7F580C2A77580FFD2A69008D3
:0B0871000593F580C2A67F0102082657
:10031B00E51075F06484E5F075F00A84FFE510755F
:10032B00F00A8485F021E4F580E516B40412E50BA0
:10033B00B40C05E4F50BB2023002057F0A75210AF5
:10034B00E4F580D2A7EF9007F393F580C2A77580F1
:10035B00FFD2A59007FE12081E120846E4F580D2C4
:10036B00A7E5219007F393F580C2A77580FFD2A56F
:10037B009007FF12081E120846E50E75F06484E51F
:10038B00F075F00A84FFE50E75F00A8485F021E51F
:10039B0016B40512E50BB40C05E4F50BB2023002F2
:1003AB00057F0A75210AE4F580D2A7EF9007F39336
:1003BB00F580C2A77580FFD2A590080012081E1207
:1003CB000846E4F580D2A7E5219007F393F580C2A8
:1003DB00A77580FFD2A590080112081E120846E5EA
:1003EB000875F06484E5F075F00A84FFE50875F094
:1003FB000A8485F021E516B40612E50BB40C05E46E
:10040B00F50BB2023002057F0A75210AE4F580D2A2
:10041B00A7EF9007F393F580C2A77580FFD2A59045
:10042B00080212081E120846E4F580D2A7E52190B7
:10043B0007F393F580C2A77580FFD2A5900803122E
:10044B00081EE4F580120846E4F580D2A7E5159066
:10045B0007F393F580C2A77580FFD2A5900804120D
:10046B00081EE4F580F580D2A7F580C2A77580FF42
:0B047B00D2A590080512081FE4F580D0
:010486002253
:10000E00E50975F06484E5F075F00A84FFE509757D
:10001E00F00A8485F021E4F580E516B40112E50BB3
:10002E00B40C05E4F50BB2023002057F0A75210A05
:10003E00E4F580C2A7D2A7EF9007F393F580C2A78D
:10004E007580FFC2A6D2A69007FEE493F580C2A6E5
:10005E007F02120826120861C2A7E4F580D2A7E536
:10006E00219007F393F580C2A77580FFD2A6900763
:10007E00FFE493F580C2A67F02120826120861E5FE
:10008E001175F06484E5F075F00A84FFE51175F0E2
:10009E000A8485F021E516B40212E50BB40C05E4D2
:1000AE00F50BB2023002057F0A75210AE4F580D203
:1000BE00A7EF9007F393F580C2A77580FFD2A690A5
:1000CE000800E493F580C2A67F021208261208618A
:1000DE00E4F580D2A7E5219007F393F580C2A775CA
:1000EE0080FFD2A6900801E493F580C2A67F02128B
:1000FE000826120861E51275F06484E5F075F00AC1
:10010E0084FFE51275F00A8485F021E516B403121A
:10011E00E50BB40C05E4F50BB2023002057F0A754F
:10012E00210AE4F580D2A7EF9007F393F580C2A7DA
:10013E007580FFD2A6900802E493F580C2A67F02D6
:10014E00120826120861E4F580D2A7E5219007F384
:10015E0093F580C2A77580FFD2A6900803E493F5AD
:10016E0080C2A6E4F5807F02120826120861E4F52B
:10017E0080D2A7F580C2A77580FFD2A690080493FF
:0C018E00F580C2A6E4F5807F020208267E
:10075C00E50924D0FFE43407AB07FAEB5403700C23
:10076C00FC7D64AE02120290ED4C700FAE02AF0332
:10077C007C017D90120290ED4C7006D200750F1E1C
:06078C0022C200750F1DE2
:010792002244
:10079300E51164016023E5116403601DE51164053F
:1007A3006017E51164076011E5116408600BE5113A
:1007B300640A6005E511B40C04750A2022750A1F4A
:0107C3002213
:1006FA00E50B6428705BF50B0508E508643C70514E
:10070A00F508050EE50E643C7047F50E0510E51078
:10071A006418703DF51005121204898F151207939B
:10072A00E51164026021E512650A7025751201055A
:10073A00111204898F15E511640D701575110112D6
:10074A0004878F1502075CE512B50F0575120105BE
:02075A0011226A
:03000B0002089C4C
:09089C00758C4C758A00050B32C5
:08081E00E493F580C2A57F02FE
:100826007E00D3EF9400EE940040147D147C00ED1E
:0F0836001D70011CED4C70F7EF1F70E61E80E384
:010845002290
:0B0487000509AF09FEAD11FCAB12FA35
:0C0492008E218F228C238D248A258B263E
:10049E0078277C007D007BFF7A0879067E007F1826
:1004AE0012026AE4FBFAF541754202F543F544E5A2
:1004BE002224D0F522E5213407F521FEAF227C005F
:1004CE007D041202E5ED4C700EAE21AF22FC7D6470
:1004DE001202E5ED4C700FAE21AF227C017D901221
:1004EE0002E5ED4C701BD3E5249402E52364809461
:1004FE0080500EE52224FFF540E52134FFF53F80C4
:10050E000685213F852240900770D3E5829522E52E
:10051E00216480F8E58364809850307C007D64AF60
:10052E0082AE831202E5ED4C60070BBB00010A8020
:10053E00147C017D90AF82AE831202E5ED4C700506
:10054E000BBB00010AA3A3A3A380BFE5402490CF59
:10055E00E53F34F8CF2542CF3541CF2BCF3AFEE5DC
:10056E002425E02425F8E6FC08E62FFFEE3CCF25F7
:10057E0026CF3525FE7C007D071202E58C438D4487
:04058E00AE43AF4485
:010592002246
:0300000002089063
:0C089000787FE4F6D8FD75814402087CF6
:10019A00E709F608DFFA8046E709F208DFFA803E47
:1001AA0088828C83E709F0A3DFFA8032E309F60834
:1001BA00DFFA8078E309F208DFFA807088828C839C
:1001CA00E309F0A3DFFA806489828A83E0A3F60850
:1001DA00DFFA805889828A83E0A3F208DFFA804C2A
:1001EA0080D280FA80C680D4806980F28033801001
:1001FA0080A680EA809A80A880DA80E280CA80336A
:10020A0089828A83ECFAE493A3C8C582C8CCC583E1
:10021A00CCF0A3C8C582C8CCC583CCDFE9DEE780B1
:10022A000D89828A83E493A3F608DFF9ECFAA9F030
:10023A00EDFB2289828A83ECFAE0A3C8C582C8CC86
:10024A00C583CCF0A3C8C582C8CCC583CCDFEADE9F
:10025A00E880DB89828A83E493A3F208DFF980CC01
:10026A0088F0EF60010E4E60C388F0ED2402B404FA
:10027A000050B9F582EB2402B4040050AF232345A1
:06028A0082239001EA73DB
:10029000BC000BBE0029EF8DF084FFADF022E4CC52
:1002A000F875F008EF2FFFEE33FEEC33FCEE9DEC1B
:1002B000984005FCEE9DFE0FD5F0E9E4CEFD22ED61
:1002C000F8F5F0EE8420D21CFEADF075F008EF2FAB
:1002D000FFED33FD4007985006D5F0F222C398FD9C
:0502E0000FD5F0EA2239
:1002E500C2D5EC30E709B2D5E4C39DFDE49CFCEE34
:1002F50030E715B2D5E4C39FFFE49EFE120290C31A
:10030500E49DFDE49CFC800312029030D507C3E414
:060315009FFFE49EFE22A2
:00000001FF
